:100000000EC015C014C013C012C011C010C00FC064
:100010000EC00DC00CC00BC00AC009C008C011241E
:100020001FBECFE5D1E0DEBFCDBF02D034C0E8CFE8
:1000300087B3896187BB18BA81E287B913B886EEA6
:1000400086B983B7846083BF2FEF89E698E121509A
:1000500080409040E1F700C0000095B1292F220FA9
:10006000392F330F330F9111C39A2111C49A3323BF
:1000700071F0C09A0CC082B7981301C0C39882B7C0
:10008000281301C0C49882B7381301C0C09882B742
:0A0090008111F1CFE2CFF894FFCF09
:00000001FF
